:10000000AB2B820700340034013401340234023453
:100010000334033404340534063407340834093413
:100020000A340B340C340E341034123414340F30C0
:10003000831201058207000000000000000000009C
:1000400000000000000000000000000000000000B0
:100050000000000079088500E23081007508840006
:100060000508F600F70A0008F800840A0008F900FD
:10007000840A4C30841E0408F500780885000800C6
:10008000C2011430420203184C284C30420784004D
:1000900083138001C20A41284C30F500F901FC307D
:1000A00081001728831603130F170F1F8F120F1BC2
:1000B0008F168F1E0F128F1A0F16FF239000083015
:1000C0008500831210100C100830831681008312F3
:1000D000101690161014191599141914850108009A
:1000E000C3000E08EB0068086B02031CE90A6B08EA
:1000F000E80043086B07EA000E086A06031D7C2827
:100100000800C200E901C830690203188F282230B4
:10011000850042087020850142087020832808006D
:10012000E901C8306902031898280A307020912824
:100130000800E801E9018E01AE308120CF30812036
:10014000902090209020CF308120C3308120AE308D
:10015000812067308120902067308120902082307C
:10016000812090209020902883120313C3008C13C9
:10017000420883169B008312430883169A001C15BD
:1001800055309D00AA309D009C141C11831203134E
:100190008C1FC628831203138C13831203130800C9
:1001A00083120313C200420883169B001C141A0812
:1001B0008312C30083120313430808000030D020C9
:1001C000ED006D082A3A031DE9280130D020ED002A
:1001D000ED28C2012A30B420ED0108001C30EE00E9
:1001E0001C30EF001C30F0001C30F1004E30F200EB
:1001F0004E30F3004E30F4000800EE1B1728172095
:10020000E208031905291C30EE00EE031720EE1F4B
:1002100012290130C2006D08B42017200A30E00016
:100220000A30E100EF1B30291720E11F1B29ED30B8
:100230006102031C1D291C30EF001720E01B24293C
:100240001430600203182D291720E01F2B29ED30F0
:100250006002031C2D291C30EF001720EF034229F8
:100260001720E01B3A2914306002031C3A296D1450
:1002700017203B296D1017201C30EF000A30E000DA
:100280000A30E1001720F01B61291720E11B4C29DF
:100290001330610203184E291C30F0001720E01BB8
:1002A00055291330600203185E291720E01F5C29CE
:1002B000EC306002031C5E291C30F0001720F003B4
:1002C00071291720E01B6B2913306002031C6B2976
:1002D000ED1417206C29ED1017201C30F000E00100
:1002E000E1011720F11B80291720E21B7B29283010
:1002F000620203187D291C30F1001720F1038D29BB
:1003000017206008F2076108F3076308F4071C3040
:10031000F1000A30E0000A30E1001720E20117285E
:100320001720FA01F70117200830050549060319BF
:10033000CA29F71F9329F701172008300505490638
:100340000319CA29F71F9C29F70117200830050552
:1003500049060319CA29F71FA529F70117200830F4
:10036000050549060319CA29F71FAE29F701172009
:100370000830050549060319CA29F71FB729F701EF
:1003800017200830050549060319CA29F71FC02997
:1003900017200134F70117200830760549060319A4
:1003A000FA0A172000341720C3010430430203184F
:1003B000142A17203430F7021720083005054906A3
:1003C000031DE629F71BDC291720013417203430E0
:1003D0007707CB001720CB1BF02905304B02031CFD
:1003E0000134C930F70717200830050549060319FD
:1003F000FD29F71BF3291720013417206A307707EE
:10040000CB00172060304307840083134B08800023
:100410000230F7001720CB1B102A32304B02031C8E
:1004200001341720C30AD52917204A08033A031DAF
:10043000222A6208CB0017206308E2004B08E30081
:100440001720003417204A0B2E2A6108CB001720F2
:100450006208E1004B08E200172000341720CA08A8
:10046000031D402A6008CB0017206108E0004B08FC
:10047000E1006108CB0017206208E1004B08E200B0
:1004800017200034172064086007E4000310E40C10
:100490006408E000172065086107E5000310E50C1B
:1004A0006508E100172066086207E6000310E60C05
:1004B0006608E200172067086307E7000310E70CEF
:1004C0006708E30017207208E0027308E1023C307D
:1004D000E2027408E3021720E21BE201FD2017206C
:1004E0006D1C782A6008CB006108E0024B08E10728
:1004F0001720E01F802AE009E00A0130E800822A84
:100500000230E8001720E11F8A2AE109E10A1030D1
:10051000E9008C2A2030E9001720E31F932AE30921
:10052000E30AEB01942AEB0117200314E21F0314E2
:10053000E21F0310E20C1720E01BA42A1530600212
:10054000031CA42A1430E0001720E11BAD2A15304B
:100550006102031CAD2A1430E1001720E21BB62A09
:1005600015306202031CB62A1430E2001720E31B88
:10057000BF2A15306302031CBF2A1430E300172082
:10058000ED1C1728172060080120E00017206108E3
:100590000120E100172063080120E3001728C501AE
:1005A000C601C701C8011720C30114304302031854
:1005B00017281720C2016008C502C51FE42A1720AA
:1005C0001430C5076808C20717206108C602C61F95
:1005D000EE2A17201430C6076908C20717206208E0
:1005E000C702C71FF82A17201430C7076A08C207B6
:1005F00017206308C802C81F022B17201430C80731
:100600006B08C20717204C3043078400831342084D
:1006100080001720C30AD52AE201EC010430EA0069
:10062000080017200C30FB0080300F07FC0008008A
:1006300017207C080F028039031D172817208030EF
:10064000FC07FB08031D4D2B17200C30FB0004306A
:10065000E0000130E80017206D1C312B0430E10070
:10066000322BE10117201030E9006C08E200043061
:10067000E300EB011720CF2217200314E21F031021
:10068000620CCB006208CB0717200314CB1F0310AA
:100690004B0CE20017206208EC00FB031728172020
:1006A0000C300F07FE0004300F07FD0017207D08F7
:1006B0000F0280390319732B1720083005054906EE
:1006C000031D712B172004300F07FD004908083C5B
:1006D000C90017207E080F028039031D712B1720D7
:1006E00001341720572B1720003417200230CA007E
:1006F00017204F23003A03197F2B1720792B9021C5
:10070000003A031D782B1720D321003A03198A2BB6
:100710001720782BE8011720C20104304202031889
:100720001728172060304207840083130008CB008D
:1007300017204E30CB02CB1F9F2BCB09CB0A1720A3
:1007400068084B02031CA82B4B08E8004208CA00AB
:100750001720C20A8D2B52209920DE200C23C001C5
:10076000EE20C901C101043041020318BF2B6430DF
:100770004107840083134E308000C10AB32B402010
:100780007523C0080319112317200430C000172057
:100790001720C008031D182317204F23003A031DFC
:1007A000EA2B17209021003A031DEA2B1720D321B2
:1007B000003A031DEA2B172042221720C008031914
:1007C000E42BC0031720C82B1720CF221720620864
:0807D000EC00C82B1720C12B1F
:0207FE000934BC
:044200002A00000090
:02400E008433F9
:00000001FF
